:100000000C942A001895000018950000189500001F
:10001000189500001895000018950000189500002C
:100020001895000018950000189500000C941B030B
:10003000189500000C94A2120C94D412189500008C
:1000400018950000189500001895000018950000FC
:10005000189500008FE58DBFCCEFECE44E2E88E0C4
:100060008EBFD7E0F7E05F2EEEEFF7E0A0E6B0E05E
:10007000A89584B7082E877F84BF88E1992781BD22
:1000800091BD88278D933197E9F788E089B980E0A1
:1000900080BD88E18AB9662480E08ABB80E087BBA6
:1000A000BC9ABB9ABA9A8FEF84BB8FEF81BB8A98B8
:1000B00087E886B980E087B9379A85E083BF81EB0E
:1000C0008FBD81E08EBD8FEF8ABD579A0E94CB1302
:1000D000A7E4B1E0E0EAF7E20E94E210A9E4B1E0AF
:1000E000E2EAF7E20E94E210ABE4B1E0E4EAF7E210
:1000F0000E94E210AFE4B1E0E8EAF7E20E94E21009
:10010000A3E5B1E0ECEAF7E20E94E210A7E5B1E076
:10011000E0EBF7E20E94E210ABE5B1E0E4EBF7E2DE
:100120000E94E210AFE5B1E0E8EBF7E20E94E210D6
:10013000A3E6B1E0ECEBF7E20E94E210A7E6B1E043
:10014000E0ECF7E20E94E210ABE6B1E0E4ECF7E2AB
:100150000E94E210AFE6B1E0E8ECF7E20E94E210A4
:10016000A3E7B1E0ECECF7E20E94E210A7E7B1E010
:10017000E0EDF7E20E94E21081E080937B0182E0F3
:1001800080937C0183E080937D0184E080937E01F5
:1001900085E080937F0186E08093800187E08093F3
:1001A000810188E08093820189E0809383018AE065
:1001B000809384018BE0809385018CE0809386019D
:1001C0008FEF8ABD80E088BD00EE14EB27E039E0B8
:1001D000ACE9B1E00D931D932D933C9380E08093A7
:1001E000CE0184E690E0A4EEB1E08D939C93C29A98
:1001F00086E990E00E94A610C39A86E990E00E94EA
:10020000A610C49A8AEF90E00E94A610C298C398E4
:10021000C49880E090E0A2E9B1E08D939C9301E066
:1002200010E020E030E0A8EAB1E00D931D932D939B
:100230003C934AE050E060E070E0A8EAB1E00D9144
:100240001D912D913C910E9405131CF011F00C940E
:100250004901A2E9B1E00D911C910F931F9307B1E1
:10026000007E076007B90E94E810482F592F1F91A0
:100270000F91040F151FA2E9B1E00D931C9381E0CB
:1002800090E00E94A610A8EAB1E00E94520F0C94E0
:100290001901A2E9B1E00D911C914AE050E00E94E1
:1002A000750FA2E9B1E04D935C9384E690E00E9463
:1002B000A610A2E9B1E00D911C91043650E015079B
:1002C0000CF402C00C94690184E08093E6010C9464
:1002D000E6080E94DD0A789489B7816089BF0091A1
:1002E0003B01013011F00C94A30180E080933B01AD
:1002F000A6EBB0E03FE30E94BE0FA6EBB0E08C910E
:10030000082F0A3011F00C94A101A6EBB0E00E9476
:10031000B113082F41E0041BACE3B1E00C93A6EB52
:10032000B0E00E94B113EA2FFB2F00913C013197FE
:10033000E01BF0400FEFA6EBB0E00E94A9130C9475
:100340007D010E94520C00914601013011F00C9485
:100350005B028BE10E940D10E4EDF7E20E940310B6
:100360008BE10E940D10EAEDF7E20E940310EEED22
:10037000F7E20E9403100E940A10E6EFF7E20E94E3
:1003800003100E940A10EEE0F8E20E940310A4E3BA
:10039000B7E0E0EBF1E00E941B130E94FB0F0E940C
:1003A0000A10EAE1F8E20E940310A4E3B7E0E6ECE9
:1003B000F1E00E941B130E94FB0F0E940A10E4E26E
:1003C000F8E20E940310A4E3B7E0E3EDF1E00E943D
:1003D00020130E94FB0F0E940A10E0E3F8E20E9443
:1003E0000310A4E3B7E0E2E9F1E00E9420130E94C9
:1003F000FB0F0E940A10E0E4F8E20E940310A4E35D
:10040000B7E0E0E9F1E00E9420130E94FB0F0E9498
:100410000A10EEE4F8E20E940310A4E3B7E0E4EB74
:10042000F1E00E9420130E94FB0F0E940A10EEE5EB
:10043000F8E20E940310A4E3B7E0E6EBF1E00E94CB
:1004400020130E94FB0F0E940A10E0E7F8E20E94CE
:100450000310A4E3B7E0EAECF1E00E941B130E9452
:10046000FB0F0E940A10EAE7F8E20E940310A4E3DF
:10047000B7E0E6EEF1E00E9427130E94FB0F0E9416
:100480000A10E6E8F8E20E940310A4E3B7E0EEECFD
:10049000F1E00E9427130E94FB0F0E940A10E0E97E
:1004A000F8E20E9403100E940A1088EC90E00E947B
:1004B000A6100C94190384E190E00E94A610E4E9D0
:1004C000F8E20E940310A4E3B7E0E0EBF1E00E9441
:1004D0001B130E94FB0F0E940A1084E190E00E940F
:1004E000A610EAE9F8E20E940310A4E3B7E0E6EC04
:1004F000F1E00E941B130E94FB0F0E940A1084E18E
:1005000090E00E94A610E0EAF8E20E940310A4E343
:10051000B7E0E3EDF1E00E9420130E94FB0F0E9480
:100520000A1084E190E00E94A610E6EAF8E20E9438
:100530000310A4E3B7E0E2E9F1E00E9420130E9477
:10054000FB0F0E940A1084E190E00E94A610ECEAE2
:10055000F8E20E940310A4E3B7E0E0E9F1E00E94B2
:1005600020130E94FB0F0E940A1084E190E00E9479
:10057000A610E2EBF8E20E940310A4E3B7E0E4EB7C
:10058000F1E00E9420130E94FB0F0E940A1084E1F8
:1005900090E00E94A610E8EBF8E20E940310A4E3AA
:1005A000B7E0E6EBF1E00E9420130E94FB0F0E94EF
:1005B0000A1084E190E00E94A610EEEBF8E20E949F
:1005C0000310A4E3B7E0EAECF1E00E941B130E94E1
:1005D000FB0F0E940A1084E190E00E94A610E4EC58
:1005E000F8E20E940310A4E3B7E0E6EEF1E00E9417
:1005F00027130E94FB0F0E940A1084E190E00E94E2
:10060000A610EAECF8E20E940310A4E3B7E0EEECD7
:10061000F1E00E9427130E94FB0F0E940A1084E160
:1006200090E00E94A610E0E9F8E20E9403100E9408
:100630000A100C946F010F921F922F923F924F92CB
:100640005F927F92AF92BF920F931F932F933F932E
:100650004F935F936F937F938F939F93AF93BF93CA
:10066000CF93DF93EF93FF938FB78F9384E68093BD
:1006700052000E9419090E94AC040E94E4030E94E7
:1006800088050E945F038F918FBFFF91EF91DF91EB
:10069000CF91BF91AF919F918F917F916F915F911A
:1006A0004F913F912F911F910F91BF90AF907F90ED
:1006B0005F904F903F902F901F900F901895A4EB54
:1006C000B1E00D911C91043B50E015071CF011F0B6
:1006D0000C946C030C94720384EB90E0A4EBB1E0F7
:1006E0008D939C93A4EBB1E00D911C910C345FEFC2
:1006F00015070CF402C00C9483038CE49FEFA4EB69
:10070000B1E08D939C93A6EBB1E00D911C91043B5D
:1007100050E015071CF011F00C9490030C94960314
:1007200084EB90E0A6EBB1E08D939C93A6EBB1E057
:100730000D911C910C345FEF15070CF402C00C9462
:10074000A7038CE49FEFA6EBB1E08D939C93A4EB01
:10075000B1E00D911C91003050E015070CF402C07F
:100760000C94B503969A0C94B6039698A6EBB1E058
:100770000D911C91003050E015070CF402C00C9450
:10078000C403979A0C94C5039798A4EBB1E08D919C
:100790009C910E94950FA0EAB1E08D939C93A6EBEB
:1007A000B1E08D919C910E94950FA2EAB1E08D93EA
:1007B0009C930FEF4091A001041B0ABDA2EAB1E097
:1007C0008C9188BD08950895A0EBB1E00D911D9125
:1007D0002D913C91A8EAB1E00D931D932D933C938C
:1007E000A8EAB1E00D911D912D913C9141E150E0BD
:1007F00060E070E00E94BF10A8EAB1E00D931D9385
:100800002D933D93A6ECB1E00D911D912D913C915E
:1008100041E150E060E070E00E94BF10A4EAB1E066
:100820000D931D932D933D93A4EAB1E00D911D917D
:100830002D913C91A8EAB1E04D915D916D917C9133
:100840000E94FB12AAECB1E00D931D932D933D93F2
:10085000AFECB1E00D911D912D913C91AAECB1E06E
:100860004D915D916D917C910E94FB12AFECB1E0D6
:100870000D931D932D933D9348ED56ED60E070E090
:10088000AFECB1E00D911D912D913C910E940513AB
:100890001CF011F00C944E040C94580408ED16ED65
:1008A00020E030E0AFECB1E00D931D932D933C932D
:1008B00048E259E26FEF7FEFAFECB1E00D911D918F
:1008C0002D913C910E9405130CF402C00C9472040B
:1008D00008E219E22FEF3FEFAFECB1E00D931D936B
:1008E0002D933C93AFECB1E00D911D912D913C9176
:1008F0004BE950E060E070E00E943E10A8EAB1E0F1
:100900004D935D936D937D93AAECB1E00D911D9194
:100910002D913C9145EA50E060E070E00E943E106D
:10092000A4EAB1E04D935D936D937D93A8EAB1E0A5
:100930000D911D912D913C91A4EAB1E04D915D91F5
:100940006D917C910E94FB12AAEBB1E00D931D9377
:100950002D933D930895089500E010E020E030E0ED
:10096000A4EAB1E00D931D932D933C9340E050E039
:1009700060E070E0AFECB1E00D911D912D913C91E4
:100980000E9405131CF011F00C94C8040C94DA04B6
:10099000AFECB1E00D911D912D913C9140E25EE4F0
:1009A00060E070E00E940013A4EAB1E00D931D9393
:1009B0002D933D93A4EAB1E00D911D912D913C91B1
:1009C00046E450E060E070E00E943E10A4EAB1E02E
:1009D0004D935D936D937D9380E090E0A7EEB1E041
:1009E0008D939C934DE050E060E070E0A4EAB1E0AC
:1009F0000D911D912D913C910E9405131CF011F059
:100A00000C9404050C940E050DE010E020E030E09D
:100A1000A4EAB1E00D931D932D933C9340E050E088
:100A200060E070E0A4EAB1E00D911D912D913C9140
:100A30000E9405130CF402C00C94280500E010E09D
:100A400020E030E0A4EAB1E00D931D932D933C9398
:100A500040E050E060E070E0A4EAB1E00D911D914B
:100A60002D913C910E9405131CF011F00C943A0555
:100A70000C944505A4EAB1E08D919C91A7EEB1E0FC
:100A80008D939C9382E080938701009187010030D1
:100A900011F00C94860548EA54EB67E070E0ACE98D
:100AA000B1E00D911D912D913C910E9405131CF018
:100AB00011F00C945D050C946005C29AC398C4981B
:100AC00048EA54EB67E070E0ACE9B1E00D911D91AC
:100AD0002D913C910E9405130CF402C00C947305F7
:100AE000C39AC498C29848E55EE667E070E0ACE956
:100AF000B1E00D911D912D913C910E9405130CF4D4
:100B000002C00C948605C398C298C49A08950895AB
:100B1000A8EBB1E00E94610FA8EBB1E00D911C9130
:100B20000A3050E015071CF011F00C9499050C9454
:100B3000A90500918701013011F00C94A205C29A19
:100B4000C39AC49A00918701023011F00C94A90550
:100B5000C49AA8EBB1E00D911C91003150E015074B
:100B60001CF011F00C94B6050C94DC050091870183
:100B7000003018F011F00C94BF050C94C705C29812
:100B8000C398C498A5EDB1E08C918F5F8C9381E000
:100B900090E0A8EBB1E08D939C930091D5010A30D1
:100BA00018F011F00C94D6050C94DC0580E08093CD
:100BB000D50180E080938701AEEDB1E00D911D91EC
:100BC00017FB1EF42FEF3FEF02C022273327A3EDC0
:100BD000B1E04D915D9157FB1EF46FEF7FEF02C0C6
:100BE000662777270E940013AAEDB1E00D931D93AD
:100BF0002D933D93AFECB1E00D911D912D913C9162
:100C000040E25EE460E070E00E943E10A4EAB1E0E1
:100C10004D935D936D937D93A4EAB1E00D911D9189
:100C20002D913C910E949210A4EAB1E00D931D9386
:100C30002D933D9341E050E060E070E0A4EAB1E024
:100C40000D911D912D913C910E9405130CF402C051
:100C50000C94340601E010E020E030E0A4EAB1E0BA
:100C60000D931D932D933C93AAEDB1E00D911D9131
:100C70002D913C91A4EAB1E04D915D916D917C91F3
:100C80000E943E10AAEDB1E04D935D936D937D936C
:100C9000AFECB1E00D911D912D913C9140ED57E0ED
:100CA00060E070E00E943E10A4EAB1E04D935D93D5
:100CB0006D937D93A4EAB1E00D911D912D913C912E
:100CC0000E949210A4EAB1E00D931D932D933D93E1
:100CD00046E150E060E070E0A4EAB1E00D911D91C2
:100CE0002D913C910E9405131CF011F00C947A0692
:100CF0000C94840606E110E020E030E0A4EAB1E0C4
:100D00000D931D932D933C930BE110E020E030E018
:100D1000A4EAB1E04D915D916D917C910E94001328
:100D2000A4EAB1E00D931D932D933D93A4EAB1E0A5
:100D30000D911D912D913C914FEF5FEF6FEF7FEF84
:100D40000E94BF10ACEAB1E00D931D932D933D932B
:100D5000A4EAB1E04D915D916D917C91AAEDB1E075
:100D60000D911D912D913C910E9405131CF011F0E5
:100D70000C94BC060C94C806A4EAB1E00D911D9138
:100D80002D913C91AAEDB1E00D931D932D933C93D1
:100D9000ACEAB1E04D915D916D917C91AAEDB1E02D
:100DA0000D911D912D913C910E9405130CF402C0F0
:100DB0000C94E606ACEAB1E00D911D912D913C91A9
:100DC000AAEDB1E00D931D932D933C93AAEDB1E0F4
:100DD0000D911D912D913C91AEEBB1E00D931D93C2
:100DE0002D933C930027A0E3B0E08C9182FB0EF49E
:100DF00001E040E0041711F00C9406078DE790E045
:100E0000A4EEB1E08D939C930C942007A4EEB1E086
:100E10000D911C91003355E715070CF402C00C949A
:100E20001D07A4EEB1E00D911C9141E050E0040FCC
:100E3000151FA4EEB1E00D931C9381E08093870110
:100E4000AAEBB1E00D911D912D913C914DE750E041
:100E500060E070E00E94BF10AAEBB1E00D931D931B
:100E60002D933D93AAEBB1E00D911D912D913C91F5
:100E7000A4EEB1E04D915D9157FB1EF46FEF7FEF53
:100E800002C0662777270E943E10AAEBB1E04D937F
:100E90005D936D937D93AAEBB1E00D911C91AEEB48
:100EA000B1E04D915C91041B150BA4EBB1E00D93E7
:100EB0001C93AAEBB1E00D911C91AEEBB1E04D910A
:100EC0005C91040F151FA6EBB1E00D931C930091EC
:100ED000CE01003011F00C94D30780E090E0A4EB39
:100EE000B1E08D939C9380E090E0A6EBB1E08D9310
:100EF0009C9300E010E020E030E0AAEBB1E00D931D
:100F00001D932D933C9300E010E020E030E0A2EC34
:100F1000B1E00D931D932D933C9300E010E020E091
:100F200030E0AFECB1E00D931D932D933C9300E0C6
:100F300010E020E030E0A4E9B1E00D931D932D9383
:100F40003C9300E010E020E030E0A0EBB1E00D9336
:100F50001D932D933C9300E010E020E030E0A6EDDF
:100F6000B1E00D931D932D933C93A2E9B1E00D9157
:100F70001C91023350E015071CF011F00C94C207CD
:100F80000C94D1070E94DD0A81E08093CE0100E03D
:100F900010E020E030E0A6EDB1E00D931D932D931D
:100FA0003C930C94E408013011F00C945508A2E92C
:100FB000B1E00D911C91023350E015070CF402C012
:100FC0000C94530840E050E060E070E0AFECB1E01A
:100FD0000D911D912D913C910E9405130CF402C0BE
:100FE0000C94090840E050E060E070E0AFECB1E044
:100FF0000D911D912D913C910E9405130CF402C09E
:101000000C94090881E080938701A6EDB1E00E946D
:10101000520F40E050E060E070E0AFECB1E00D91C5
:101020001D912D913C910E9405131CF011F00C9420
:101030001B080C94340840E050E060E070E0AFEC36
:10104000B1E00D911D912D913C910E9405131CF072
:1010500011F00C942D080C94340881E080938701E2
:10106000A6EDB1E00E94520F40E550E060E070E074
:10107000A6EDB1E00D911D912D913C910E940513BB
:101080001CF011F00C9446080C94530883E08093F4
:10109000CE0100E010E020E030E0A6EDB1E00D93DD
:1010A0001D932D933C930C94E408033011F00C94A1
:1010B000E10801E010E020E030E0A4EAB1E00D93A7
:1010C0001D932D933C934FEF50E060E070E0A4EA55
:1010D000B1E00D911D912D913C910E9405131CF0E2
:1010E00011F00C94DC08A4EBB1E00D911C910030E0
:1010F00050E0150781E009F080E08F93A6EBB1E0A6
:101100000D911C91003050E0150781E009F080E05E
:101110009F918923882311F40C9490080C94DC0887
:10112000A4EBB1E00D911C91003050E015071CF0CC
:1011300011F00C949D080C94A108A4EBB1E00E945E
:10114000680FA4EBB1E00D911C91003050E0150741
:101150000CF402C00C94B008A4EBB1E00E94610F43
:10116000A6EBB1E00D911C91003050E015071CF08A
:1011700011F00C94BD080C94C108A6EBB1E00E94DC
:10118000680FA6EBB1E00D911C91003050E01507FF
:101190000CF402C00C94D008A6EBB1E00E94610FE1
:1011A00082E390E00E94A6100E945F03A4EAB1E0EF
:1011B0000E94520F0C94630880E08093CE010C943F
:1011C000E40883E08093CE010895089501E010E0E3
:1011D00020E030E0A8EAB1E00D931D932D933C93FD
:1011E000A6EEB1E04C91552766277727A8EAB1E033
:1011F0000D911D912D913C910E9405131CF011F051
:101200000C941209C49A86E990E00E94A610C49832
:1012100086E990E00E94A610A8EAB1E00E94520F71
:101220000C94F008E2E0F0E00E9435100C94E6081F
:10123000089507B1007E056007B90E94E810ACE888
:10124000B1E08D939D9388278D938C9300E014E0FB
:1012500020E030E0ACE8B1E04D915D916D917C9182
:101260000E940013ACE8B1E00D931D932D933D93C4
:1012700007B1007E036007B90E94E810A8E8B1E05A
:101280008D939D9388278D938C9307B1007E00608A
:1012900007B90E94E810A0E9B1E08D939C9307B1D3
:1012A000007E066007B90E94E810A3EDB1E08D93BF
:1012B0009C9300E014E00F931F9307B1007E07603A
:1012C00007B90E94E810482F592F1F910F91041B56
:1012D000150BA2E9B1E00D931C93A4E9B1E00D91C7
:1012E0001D912D913C914CE251E060E070E00E9434
:1012F0003E10A8EAB1E04D935D936D937D93A4E910
:10130000B1E00D911D912D913C91A8EAB1E04D9174
:101310005D916D917C910E940013A4E9B1E00D9361
:101320001D932D933D93A8E8B1E00D911D912D9152
:101330003C91A0EEB1E04D915C91662777270E9429
:101340000013A8EAB1E00D931D932D933D93A8EAF5
:10135000B1E00D911D912D913C91A7EEB1E04D9121
:101360005D9157FB1EF46FEF7FEF02C06627772772
:101370000E94FB12A8EAB1E00D931D932D933D93BB
:10138000A4E9B1E00D911D912D913C91A8EAB1E045
:101390004D915D916D917C910E94FB12A4E9B1E0A9
:1013A0000D931D932D933D93A8E9B1E00D911D91EF
:1013B0002D913C914CE251E060E070E00E943E10C3
:1013C000A4EAB1E04D935D936D937D93A8E9B1E0FC
:1013D0000D911D912D913C91A4EAB1E04D915D914B
:1013E0006D917C910E940013A8E9B1E00D931D93CB
:1013F0002D933D93A8E9B1E00D911D912D913C9164
:10140000ACE8B1E04D915D916D917C910E94FB1231
:10141000A8E9B1E00D931D932D933D93A8E9B1E0A8
:101420000D911D912D913C914EE150E060E070E0F6
:101430000E943E10A4EAB1E04D935D936D937D93BD
:10144000ACE8B1E00D911D912D913C914AE050E046
:1014500060E070E00E94BF10A8EAB1E00D931D9318
:101460002D933D93A4EAB1E00D911D912D913C91F6
:10147000A8EAB1E04D915D916D917C910E940013BD
:10148000A4EAB1E00D931D932D933D93A4EAB1E03E
:101490000D911D912D913C9143E250E060E070E090
:1014A0000E94BF10A4EAB1E00D931D932D933D93CC
:1014B000A4EAB1E00D911D912D913C9144E650E0DC
:1014C00060E070E00E943E10A4EAB1E04D935D93AD
:1014D0006D937D93A4EAB1E00D911D912D913C9106
:1014E000A6ECB1E00D931D932D933C93A4E9B1E0DC
:1014F0000D911D912D913C91A6ECB1E04D915D9126
:101500006D917C910E94FB12A4E9B1E00D931D93B3
:101510002D933D93A4E9B1E00D911D912D913C9146
:101520004EE150E060E070E00E943E10A0EBB1E0C0
:101530004D935D936D937D93ACE9B1E00D911D9159
:101540002D913C914CE251E060E070E00E943E1031
:10155000A4EAB1E04D935D936D937D93ACE9B1E066
:101560000D911D912D913C91A4EAB1E04D915D91B9
:101570006D917C910E940013ACE9B1E00D931D9335
:101580002D933D93ACE9B1E00D911D912D913C91CE
:10159000A0E9B1E04D915D9157FB1EF46FEF7FEF35
:1015A00002C0662777270E94FB12ACE9B1E00D93D9
:1015B0001D932D933D930895089580E090E0A3ED51
:1015C000B1E08D939C9301E010E020E030E0A8EAC8
:1015D000B1E00D931D932D933C934AE050E060E001
:1015E00070E0A8EAB1E00D911D912D913C910E940F
:1015F00005131CF011F00C941D0BA3EDB1E00D913F
:101600001C910F931F9307B1007E066007B90E94DB
:10161000E810482F592F1F910F91040F151FA3EDAC
:10162000B1E00D931C9381E090E00E94A610A8EA1F
:10163000B1E00E94520F0C94ED0AA3EDB1E00D91C0
:101640001C914AE050E00E94750FAEEDB1E04D9361
:101650005C9300E010E020E030E0ACE8B1E00D93F6
:101660001D932D933C9301E010E020E030E0A8EAC8
:10167000B1E00D931D932D933C9344E650E060E060
:1016800070E0A8EAB1E00D911D912D913C910E946E
:1016900005131CF011F00C948A0B07B1007E056055
:1016A00007B90E94E810A4EAB1E08D939D938827C2
:1016B0008D938C9300E014E020E030E0A4EAB1E0E8
:1016C0004D915D916D917C910E940013A4EAB1E06F
:1016D0000D931D932D933D93ACE8B1E00D911D91B9
:1016E0002D913C91A4EAB1E04D915D916D917C9179
:1016F0000E94FB12ACE8B1E00D931D932D933D9336
:1017000082E090E00E94A610A8EAB1E00E94520F89
:101710000C943D0BACE8B1E00D911C9144E650E017
:101720000E949B0FA2EEB1E04D935C930CE211E09E
:1017300020E030E0A2EEB1E04D915C916627772782
:101740000E94BF10A8E9B1E00D931D932D933D9326
:1017500000E010E020E030E0A8E8B1E00D931D9338
:101760002D933C9301E010E020E030E0A8EAB1E0E6
:101770000D931D932D933C9344E650E060E070E0A0
:10178000A8EAB1E00D911D912D913C910E940513A5
:101790001CF011F00C94F70B07B1007E036007B941
:1017A0000E94E810A4EAB1E08D939D9388278D9361
:1017B0008C93A8E8B1E00D911D912D913C91A4EA84
:1017C000B1E04D915D916D917C910E94FB12A8E872
:1017D000B1E00D931D932D933D9382E090E00E9424
:1017E000A610A8EAB1E00E94520F0C94BC0BA8E826
:1017F000B1E00D911C9144E650E00E949B0FA0EED9
:10180000B1E04D935C93A0EEB1E00D911C910039D5
:1018100051E0150710F00C94120C83E08093E60160
:101820000C94E608A0EEB1E00D911C91083552E051
:10183000150718F011F00C941F0C0C94240C83E085
:101840008093E6010C94E608A2EEB1E00D911C91A4
:101850000E3551E0150710F00C94330C82E08093A4
:10186000E6010C94E608A2EEB1E00D911C910E3E4B
:1018700052E0150718F011F00C94400C0C94450C34
:1018800082E08093E6010C94E6080895089581E0D3
:1018900080933B010895A6EBB0E00E94FD0F0E94EB
:1018A0000A100895A6EBB0E08C91082F033211F0D6
:1018B0000C945E0C0E944B0C0C94DB0CA6EBB0E07D
:1018C0008C91082F0B3111F00C946A0C0E944B0C78
:1018D0000C94DB0CA6EBB0E0E0EAF7E22FEF91E02E
:1018E0000E94F610A5E4B1E00C9300914501003090
:1018F00018F011F00C947E0C0C94CB0CA6EBB0E01D
:10190000E0EDF8E22FEF91E00E94F610002F00309A
:1019100080E010F009F081E08F9340914501A6EB43
:10192000B0E0E0EDF8E22FEF91E00E94F610002F1A
:10193000041781E008F080E09F918923882311F447
:101940000C94AA0C0E944B0C0E94DC0C0C94DB0C37
:101950000C94C90CE6EBF0E000914501A6EFB0E075
:101960000E94A913A6EFB0E00E947113ADE3B1E0AD
:101970000C9300913D01003011F00C94C50C0E94B5
:10198000DC0C0C94DB0C0C94C90C0E944B0C0C94DA
:10199000DB0C0C94DB0C00913D01003011F00C9439
:1019A000D70C0E94DC0C0C94DB0C0C94DB0C0E941A
:1019B0004B0C0C94DB0C089581E08093EA01A6EFB8
:1019C000B0E088278C93A6E3B1E088278C93A0E44D
:1019D000B1E0ECE9F7E20E948E1280E090E0AEE325
:1019E000B1E08D939C93A6EBB0E00E94B113082F59
:1019F0000F93A6EBB0E0E7E4F1E0222791E00E942C
:101A0000F610402F0F91041BA5E4B1E00C93A6EB58
:101A1000B0E00E94B113EA2FFB2F009145013197EE
:101A2000E01BF0400FEFA6EFB0E00E94A91381E0A9
:101A30008093E9010091E901043018F011F00C9451
:101A4000950D81E4482FA9EEB1E0AD90BB24A5EF40
:101A5000B0E0AA0DBB1D0C91041781E008F480E0F2
:101A60008F938AE5482FA9EEB1E0AD90BB24A5EF96
:101A7000B0E0AA0DBB1D0C91041781E010F009F035
:101A800080E09F9189238F9381E6482FA9EEB1E0F2
:101A9000AD90BB24A5EFB0E0AA0DBB1D0C910417BF
:101AA00081E008F480E09F91892B8F938AE7482F8B
:101AB000A9EEB1E0AD90BB24A5EFB0E0AA0DBB1D2F
:101AC0000C91041781E010F009F080E09F918923C8
:101AD000882311F40C948D0DA9EEB1E0AD90BB24D8
:101AE000A5EFB0E0AA0DBB1D8C91AAEEB1E0AD90C0
:101AF000BB24A5E3B1E0AA0DBB1D8C93AAEEB1E017
:101B00008C918F5F8C9380E0AAEEB1E0AD90BB2406
:101B1000A5E3B1E0AA0DBB1D8C93A9EEB1E08C91B9
:101B20008F5F8C9310F40C941A0DA6E3B1E00E9421
:101B3000B113082F033011F00C94D90DE6E3F1E056
:101B4000A6E3B1E00E94961280E08093E901009143
:101B5000E901093118F011F00C94D90DE9EEF1E02A
:101B60000191112744E050E00E94B510E7E4F1E054
:101B7000E00FF11FA6E3B1E00E94B91311F00C943D
:101B8000D10DA9EEB1E0AD90BB24AAE7B1E0AA0D5A
:101B9000BB1D8C91AEE3B1E08D9388278C930C94A0
:101BA000D90DA9EEB1E08C918F5F8C9310F40C9459
:101BB000A70D81E08093EA01A6E3B1E088278C932A
:101BC000A6EFB0E0E9E4F1E0222791E00E94F610F0
:101BD000A5E4B1E00C9300914501003011F00C94A4
:101BE000F80DA6EFB0E00E94B113A5E4B1E08C932C
:101BF00081E08093E901409145010091E9010417DA
:101C000018F011F00C94530E80E3482FA9EEB1E0C8
:101C1000AD90BB24A5EFB0E0AA0DBB1D0C9104173D
:101C200081E008F480E08F9389E3482FA9EEB1E0CA
:101C3000AD90BB24A5EFB0E0AA0DBB1D0C9104171D
:101C400081E010F009F080E09F918923882311F44E
:101C50000C944B0EA9EEB1E0AD90BB24A5EFB0E023
:101C6000AA0DBB1D8C91AAEEB1E0AD90BB24A5E3FB
:101C7000B1E0AA0DBB1D8C93AAEEB1E08C918F5FF1
:101C80008C9380E0AAEEB1E0AD90BB24A5E3B1E077
:101C9000AA0DBB1D8C93A9EEB1E08C918F5F8C9344
:101CA00010F40C94FB0DAEE3B1E00D911C910F9379
:101CB0001F93A6E3B1E00E947113402F512F1F9193
:101CC0000F91040F151FAEE3B1E00D931C93A6EF27
:101CD000B0E0E9E4F1E0222791E00E94F610002F45
:101CE000003018F011F00C94770E0C947E0E809159
:101CF00044018F77809344010C94830E80914401BA
:101D0000806880934401A6EFB0E00E94B113082FD1
:101D10000F93A6EFB0E0E9E4F1E0222791E00E9402
:101D2000F610402F0F91041BA5E4B1E00C93A6EF31
:101D3000B0E00E94B113EA2FFB2F009145013197CB
:101D4000E01BF0400FEFA6EFB0E00E94A913A6EF52
:101D5000B0E00E94BA11EDE0F0E0A0E4B1E00E9432
:101D6000A313AEE3B1E00D911C91013050E01507D3
:101D700011F00C94D50EA6EBB0E0E2EDF8E20E9473
:101D8000E210A6EBB0E00E94B50FE8E8F1E00E9497
:101D90001B13A6EBB0E00E94B50FEAEDF8E20E943B
:101DA000E2100E944B0C0C94510F023050E01507CA
:101DB00011F00C94F50EA6EBB0E0ECEDF8E20E9409
:101DC000E210A6EBB0E00E94B50FECE8F1E00E9453
:101DD0001B13A6EBB0E00E94B50FEAEDF8E20E94FB
:101DE000E2100E944B0C0C94510F033050E0150789
:101DF00011F00C94050FA6EBB0E0E4EEF8E20E94BF
:101E0000E2100E944B0C0C94510F043050E0150767
:101E100011F00C941E0F81E0809346018BE10E942B
:101E20000D10E4EDF7E20E9403108BE10E940D100B
:101E3000EAEDF7E20E9403100C94510F053050E0D8
:101E4000150711F00C94290F80E0809346010C9443
:101E5000510F063050E0150711F00C94490FA6EB16
:101E6000B0E0E0E1F9E20E94E210A6EBB0E00E94EF
:101E7000B50FE0E9F1E00E942013A6EBB0E00E946C
:101E8000B50FEAEDF8E20E94E2100E944B0C0C94B0
:101E9000510FA6EBB0E0E8E1F9E20E94E2100E94E7
:101EA0004B0C08950D911D912D913C9181E0080FEF
:101EB0008827181F281F381F3C932E931E930E93BC
:101EC0000895ED91FC91EF5FFF4FFC93EE93089521
:101ED000ED91FC91E150F040FC93EE93089509D010
:101EE0000E94B51000FC10D0089503D024D001F852
:101EF000F9CF0024E89457FF02C009D0689400F895
:101F00000BD010F80124089502D009D008955095FF
:101F100040954F5F5F4F0895E89417FF089500952F
:101F200010950F5F1F4F6894089599231AF48095B8
:101F3000909501960895352F242FE894452B11F4A0
:101F400068940895512F402F0027112780E1440FF6
:101F5000551F001F111F021B130B416018F4020FC5
:101F6000131F4E7F8A9599F708958F938D9188233B
:101F7000E9F711978F910895A4E3B7E018D088305E
:101F800091F08D3039F03323C9F38D933A9563FE88
:101F900044D0F4CF63FC04C08DE03FD08AE03DD054
:101FA00088278C93089539D011973395E7CF0F92F6
:101FB0009F93AF93BF937F9380918A008823E1F32F
:101FC000F89480918A008A9580938A009091880085
:101FD000A0E6B0E0A90F0024B01D8C919395983233
:101FE00009F499279093880078947F91BF91AF91DD
:101FF0009F910F900895A4E3B7E08D91882311F08D
:102000000CD0FBCF08950E94B611802D11F005D0A1
:10201000FACF08958DE001D08AE09F939FB79F93F8
:10202000AF93BF930F937F939091B5009832E1F3F4
:10203000F8949091B50093959093B50099270091ED
:10204000B400ABE8B0E0A00FB91F8C930395083241
:1020500009F400270093B400559A7F910F91BF9126
:10206000AF919F919FBF9F91089588EE93E06ED0AE
:102070003197D9F7089500FC05D0089530D005D0E8
:1020800001F8F9CF37D03FD00895842F952FA62F90
:10209000B72FE894452B462B472B11F468940895ED
:1020A000402F512F622F732F00271127222733270C
:1020B000F0E2440F551F661F771F001F111F221FDC
:1020C000331F081B190B2A0B3B0B416028F4080F28
:1020D000191F2A1F3B1F4E7FFA9559F708950024B8
:1020E000E89477FF02C006D0689400F809D010F891
:1020F0000124089512D04F5F5F4F6F4F7F4F0895B7
:10210000E89437FF089500951095209530950F5F5E
:102110001F4F2F4F3F4F68940895409550956095FD
:102120007095089537FF0895009510952095309586
:102130000F5F1F4F2F4F3F4F08953197F1F70895CD
:10214000689462F80895E89462F80895EF93FF9315
:10215000EE27E82BE92B31F0E0EAFFE03197F1F7C9
:102160000197D1F7FF91EF9108950F92B801469F23
:102170008001479F100D569F100D0F9008950F92EC
:102180001F922F92C801D901489F80014A9F900158
:102190004B9F202C499F100D211D321D5A9F202C32
:1021A000589F100D211D321D599F200D311D689F14
:1021B000200D311D699F300D789F300D2F901F909D
:1021C0000F9008950E94B6110D920020D9F708953E
:1021D000369A3699FECF369A3699FECF84B195B1AC
:1021E000089599910027A90FB01F1197492F4A957B
:1021F0005E2F6F2FE89411274395203019F0C89572
:10220000802D01C080818823B9F07C917723A1F0D3
:10221000781739F40EF0042F1395689411963196BF
:10222000EBCF112321F0411BA11B1127B10BE89427
:10223000E52FF62F1196E0CF882311F0002708959F
:102240000895D190E190F1900191089521913191FB
:10225000419151910895102F90E8FF0C001F09271C
:10226000990FF7941078652F90E8440F551F592760
:10227000990F4795607800380895FF0C90E89027F3
:10228000110F9795F794092F0895502F2D2D3E2D5E
:102290004F2D612F08952DEC3CEC4CEC5DE366274F
:1022A0000FC0CFDFF2DFDD24EE2490E8F92E0FE33C
:1022B00007C0CCDF05C02227332740E251E4662760
:1022C000552351F1002381F1C6DF71F11627005823
:1022D00050580894050B18F407FD03C025C007FDEE
:1022E00023C0469537952795F694E794D79422D046
:1022F000FF202AF0DD0CEE1CFF1C015073F09D2D19
:10230000969548F0DD203AF4EE202AF491E0D90EBB
:102310009927E91EF91EB1CF07C09FE7092FF92AB7
:102320009FEFD92EE92E0895DD24EE24FF24002707
:10233000112708959F929924AA24BB2488E1D216DC
:10234000E306F40628F0D21AE30AF40A089401C05E
:102350008894991CAA1CBB1CDD0CEE1CFF1C8A95E2
:1023600071F7D92CEA2CFB2C9F900895C8953196D3
:10237000002008950E94A310E89488278A938A93E6
:10238000D3DF11278D918032E9F31197BBD098F0FC
:102390008D3229F4109511968C91B4D060F08E3264
:1023A00029F411968C91AED008F446C022960E9472
:1023B000A01081E008958C91A5D0D8F547D0119652
:1023C000D0F703958D919ED0E0F38E3229F48C9155
:1023D00099D010F41196FBCF853419F0853609F0A9
:1023E00055C011968C918ED060F08D3219F08B32E1
:1023F00021F0DCCF08800094088211968C9182D065
:10240000A8F68053898311968C917CD058F49981D9
:10241000990F990F0980900D990F8053890F898327
:10242000873220F68981988199230AF48195080FD3
:102430002DC08E3289F611968C9164D068F606D044
:1024400018F011960A95F8CF1196C1CF4F2D3E2D59
:102450002D2DDD0CEE1CFF1CA8F0DD0CEE1CFF1C6E
:1024600088F0D20EE31EF41E68F0DD0CEE1CFF1C9B
:1024700048F0805309F06894D80E8827E81EF81EAB
:1024800008F00895F42EE32ED22E089534D019F1D9
:1024900016F5098308E921D00695882787959F2D91
:1024A0009F77980FF92E0150000F110F0795898122
:1024B000882379F01AF48195898306C0ECDE89813E
:1024C0008A958983D9F705C0F6DE89818A95898343
:1024D000D9F72296089528DFFCCF0DD041F0FF20D8
:1024E00032F00A9531F0DD0CEE1CFF1CD2F7889417
:1024F00008950894089500240D280E280F28002A16
:1025000000200895803320F08A3310F40894089551
:102510008894089591E005C092E003C094E001C062
:1025200098E024DF0D929A95E1F70895819104D007
:102530008D938823D9F70895813618F08B3708F4E6
:102540008F7D08957F930F93AF93BF938F939F9346
:102550008FB78F93E89480918A0008E2081B21F4DA
:102560009CB10E94A01013C000918900A0E6B0E0C9
:1025700077279CB1A00FB71F9C9368948395809395
:102580008A000395083209F40027009389009D30E2
:1025900011F40E94470C8F918FBF9F918F91BF9133
:1025A000AF910F917F9118957F93AF93BF938F93C6
:1025B0009F938FB78F939091B500992399F09A9537
:1025C0009093B5009927ABE8B0E08091B300A80FD5
:1025D000B91F9C918395883209F488278093B300B2
:1025E0009CB901C055988F918FBF9F918F91BF91DA
:1025F000AF917F911895040F151F261F371F08955F
:10260000041B150B260B370B089504171507260717
:1026100037070895000F111F221F331F08950095DB
:102620001095209530950F5F1F4F2F4F3F4F089506
:10263000019110810EC001911191219130810BC047
:102640000191108117FF05C03FEF2FEF04C00081FB
:1026500011272227332737FF03C0E1DF8DE28D9357
:10266000CF93DF93CF92DF92EF92AA24BB24CC24A6
:10267000DD24EE2440E2CAE0DD2755E093E38881C3
:10268000890F87FD9F7083FD907F891B89935A95E1
:10269000A9F7C0DFAA1CBB1CCC1CDD1CEE1C4A9594
:1026A00051F7E894EFE0FF2782910ED0EB30E0F78E
:1026B0001EF068948A2D0CD088278D93EF90DF90C0
:1026C000CF90DF91CF910895982F829501D0892FD7
:1026D0008F70805D26F0803309F4089568948D939F
:1026E000089500271127222733271DD08A3328F485
:1026F000803318F005D015D0F9CF0EF490CF08959F
:1027000080538F93402F512F622F732F83DF82DFEF
:1027100072DF80DF8F919927080F191F291F391F3A
:1027200008958D910895E894FCDF8032E9F38B32AF
:10273000D9F38930C9F38D3211F46894F2CF08953A
:1027400088278D93089594E081918D939A95E1F770
:10275000089581918D930A9519F08823D1F70895F2
:10276000EFCF8FEF83959D919923E1F708956894BA
:1027700001C0E894AF93BF938D9116F0919103C07F
:102780000E94B611902D891718F011F48823A1F733
:10279000BF91AF910895689463F808950000000018
:1027A0003A003D00414458004944470049444E0026
:1027B00054454C0053545000535749004241540073
:1027C0004D4F41004D4F420053545200455252006C
:1027D0004D4F44005B313B3166005B324A0023546D
:1027E000656C656D65747269652076312E302020C8
:1027F0002020202000002320202020202020202016
:102800002020202020202020202020200000234ED7
:10281000656967756E67203D2000234779726F20D8
:102820003D200000234C656E6B6572203D2000004A
:10283000234675DF736368616C746572203D200008
:10284000234261747465726965203D200000234D48
:102850006F746F72206C696E6B73203D2000234D86
:102860006F746F7220726563687473203D2000007E
:102870002353747265DF203D2000234665686C6534
:1028800072203D200000234D6F647573203D2000B1
:10289000313A3400323A313D0000323A333D0000E3
:1028A000323A353D0000323A363D0000323A373D8B
:1028B0000000323A383D0000323A393D0000323AE9
:1028C00031303D00323A31313D00323A31323D0053
:1028D0002A0023303A4144583D00210023303A4930
:1028E00044473D0023303A49444E3D5B4350552D0B
:1028F0004D6F64756C2076332E32206265746120D2
:1029000047FC6E746572204765726F6C645D2100D0
:1029100023303A4241543D0023303A4552523D5B08
:1029200053796E746178204572726F725D21000078
:00000001FF
